:1000000010C02AC05FC028C027C026C025C024C099
:1000100023C022C021C020C01FC01EC01DC01CC0E4
:1000200034C011241FBECFE5D1E0DEBFCDBF10E04C
:10003000A0E6B0E0ECE0F3E002C005900D92A2373C
:10004000B107D9F710E0A2E7B0E001C01D92A638D1
:10005000B107E1F7FFD058C1D3CF0F931F9300E052
:1000600010E09801061717072807390759F0E7E845
:10007000F3E13197F1F700C000000F5F1F4F2F4FE2
:100080003F4FF0CF1F910F9108951F920F920FB61F
:100090000F9211248F93809172008FB91092720089
:1000A000769A8F910F900FBE0F901F9018951FBCDE
:1000B00081E08EBD08958AB38F688ABB8BB3807749
:1000C0008BBB08951F920F920FB60F9211248F933E
:1000D0009F938BB78F7E8BBF8CB59DB5969587957B
:1000E00090937400809373009F918F910F900FBE37
:1000F0000F901F901895CF93DF93F89421E030E094
:1001000001C0220F8A95EAF7F22F22BB8BB78061DC
:100110008BBF8FEF9FEF9093740080937300789460
:10012000E2E040E050E08FEF9FEFA22FA0956E98A5
:10013000000000000000F894F2BB6AB760616ABF7B
:100140006BB760616BBF90937400809373001DBCAC
:100150001CBC78946AB36A236ABBC3ECD9E02197CC
:10016000F1F700C000006AB3622B6ABB6E9A60911F
:100170007300709174006F3F7F4F69F0609173005E
:1001800070917400460F571F000000000000E150FE
:1001900071F6CA0102C08FEF9FEFDF91CF910895F2
:1001A000CF93C82FA8DF9C012F3F8FEF380789F02E
:1001B000EC2FF0E0EE0FFF1FEA58FF4F8081918196
:1001C000281B390B213080E8380730F080E090E0C0
:1001D00004C08FEF9FEF01C0C901CF910895863011
:1001E000B8F490E0FC01E459FF4F2081332727FD4C
:1001F0003095FC01EA59FF4F4081552747FD509546
:10020000FC01E05AFF4F8081992787FD909506C039
:1002100080E090E040E050E020E030E068B36B7FA9
:10022000452B11F040E001C044E0642B68BB4BB3A8
:100230004F77892B11F080E001C080E8482B4BBB41
:100240008BB38F7D232B11F090E001C090E2892BBE
:100250008BBB0895F89480E886BD16BC8FEF81BFF4
:100260002ADF25DF789480E046DF90937700809343
:10027000760081E040DF9093790080937800BA9A0D
:100280008AB3806A8ABB80E08BDFEC0181E088DF83
:100290008C0180E085DFC80FD91F81E081DF800FEE
:1002A000911F9E01CF3FD10519F010F02FEF30E0E4
:1002B0008F3F910519F010F08FEF90E0AC01420FE5
:1002C000531F4032510510F482E31CC0821B930B74
:1002D000803E2FEF920714F480E014C0803F2FEF90
:1002E000920714F481E00EC097FF02C082E00AC0BA
:1002F0008031910514F483E005C0809714F484E004
:0C03000001C085E06CDFBFCFF894FFCF98
:10030C0000000001010100010101000001010000D9
:02031C000001DE
:00000001FF
